 GetStackTraceSuspendedStress

 Timestamp is 6dc14945 (reproducible build file hash)

 Preferred load address is 0000000180000000

 Start         Length     Name                   Class
 0001:00000000 00002de0H .text$mn                CODE
 0001:00002de0 00000036H .text$mn$00             CODE
 0001:00002e16 00000092H .text$x                 CODE
 0002:00000000 000001b0H .idata$5                DATA
 0002:000001b0 00000038H .00cfg                  DATA
 0002:000001e8 00000008H .CRT$XCA                DATA
 0002:000001f0 00000008H .CRT$XCZ                DATA
 0002:000001f8 00000008H .CRT$XIA                DATA
 0002:00000200 00000008H .CRT$XIC                DATA
 0002:00000208 00000008H .CRT$XIZ                DATA
 0002:00000210 00000008H .CRT$XLA                DATA
 0002:00000218 00000008H .CRT$XLZ                DATA
 0002:00000220 00000008H .CRT$XPA                DATA
 0002:00000228 00000008H .CRT$XPZ                DATA
 0002:00000230 00000008H .CRT$XTA                DATA
 0002:00000238 00000008H .CRT$XTZ                DATA
 0002:00000240 00000000H .gehcont$y              DATA
 0002:00000240 00000000H .gfids$y                DATA
 0002:00000240 00001540H .rdata                  DATA
 0002:00001780 00000000H .rdata$CastGuardVftablesA DATA
 0002:00001780 00000000H .rdata$CastGuardVftablesC DATA
 0002:00001780 00000028H .rdata$T                DATA
 0002:000017a8 000000b8H .rdata$voltmd           DATA
 0002:00001860 00000330H .rdata$zzzdbg           DATA
 0002:00001b90 00000008H .rtc$IAA                DATA
 0002:00001b98 00000008H .rtc$IZZ                DATA
 0002:00001ba0 00000008H .rtc$TAA                DATA
 0002:00001ba8 00000008H .rtc$TZZ                DATA
 0002:00001bb0 00000004H .tls                    DATA
 0002:00001bb4 00000004H .tls$                   DATA
 0002:00001bb8 00000008H .tls$ZZZ                DATA
 0002:00001bc0 000002e0H .xdata                  DATA
 0002:00001ea0 000000dcH .edata                  DATA
 0002:00001f7c 00000064H .idata$2                DATA
 0002:00001fe0 00000018H .idata$3                DATA
 0002:00001ff8 000001b0H .idata$4                DATA
 0002:000021a8 0000045cH .idata$6                DATA
 0003:00000000 00000050H .data                   DATA
 0003:00000050 000007e8H .bss                    DATA
 0004:00000000 00000354H .pdata                  DATA

  Address         Publics by Value              Rva+Base               Lib:Object

 0000:00000000       __AbsoluteZero             0000000000000000     <absolute>
 0000:00000000       ___safe_se_handler_count   0000000000000000     <absolute>
 0000:00000000       ___safe_se_handler_table   0000000000000000     <absolute>
 0000:00000000       __arm64x_extra_rfe_table   0000000000000000     <absolute>
 0000:00000000       __arm64x_extra_rfe_table_size 0000000000000000     <absolute>
 0000:00000000       __arm64x_native_entrypoint 0000000000000000     <absolute>
 0000:00000000       __arm64x_redirection_metadata 0000000000000000     <absolute>
 0000:00000000       __arm64x_redirection_metadata_count 0000000000000000     <absolute>
 0000:00000000       __dynamic_value_reloc_table 0000000000000000     <absolute>
 0000:00000000       __enclave_config           0000000000000000     <absolute>
 0000:00000000       __guard_check_icall_a64n_fptr 0000000000000000     <absolute>
 0000:00000000       __guard_eh_cont_count      0000000000000000     <absolute>
 0000:00000000       __guard_eh_cont_table      0000000000000000     <absolute>
 0000:00000000       __guard_fids_count         0000000000000000     <absolute>
 0000:00000000       __guard_fids_table         0000000000000000     <absolute>
 0000:00000000       __guard_iat_count          0000000000000000     <absolute>
 0000:00000000       __guard_iat_table          0000000000000000     <absolute>
 0000:00000000       __guard_longjmp_count      0000000000000000     <absolute>
 0000:00000000       __guard_longjmp_table      0000000000000000     <absolute>
 0000:00000000       __hybrid_auxiliary_iat     0000000000000000     <absolute>
 0000:00000000       __hybrid_auxiliary_iat_copy 0000000000000000     <absolute>
 0000:00000000       __hybrid_code_map          0000000000000000     <absolute>
 0000:00000000       __hybrid_code_map_count    0000000000000000     <absolute>
 0000:00000000       __x64_code_ranges_to_entry_points 0000000000000000     <absolute>
 0000:00000000       __x64_code_ranges_to_entry_points_count 0000000000000000     <absolute>
 0000:00000100       __guard_flags              0000000000000100     <absolute>
 0000:00000000       __ImageBase                0000000180000000     <linker-defined>
 0001:00000000       ?NewObject@JNIEnv_@@QEAAPEAV_jobject@@PEAV_jclass@@PEAU_jmethodID@@ZZ 0000000180001000 f i libGetStackTraceSuspendedStress.obj
 0001:00000024       ?SetEventNotificationMode@_jvmtiEnv@@QEAA?AW4jvmtiError@@W4jvmtiEventMode@@W4jvmtiEvent@@PEAV_jobject@@ZZ 0000000180001024 f i libGetStackTraceSuspendedStress.obj
 0001:00000118       ?TranslateError@@YAPEBDW4jvmtiError@@@Z 0000000180001118 f   libGetStackTraceSuspendedStress.obj
 0001:000003d0       ?TranslateState@@YAPEBDH@Z 00000001800013d0 f   libGetStackTraceSuspendedStress.obj
 0001:00000760       ?check_link_consistency@@YAXPEAU_jvmtiEnv@@PEAUJNIEnv_@@PEAV_jobject@@@Z 0000000180001760 f   libGetStackTraceSuspendedStress.obj
 0001:0000102c       ?print_thread_info@@YAXPEAU_jvmtiEnv@@PEAUJNIEnv_@@PEAV_jobject@@@Z 000000018000202c f   libGetStackTraceSuspendedStress.obj
 0001:000013d0       Agent_OnLoad               00000001800023d0 f   libGetStackTraceSuspendedStress.obj
 0001:000015a8       Java_jdk_test_lib_jvmti_DebugeeClass_checkStatus 00000001800025a8 f   libGetStackTraceSuspendedStress.obj
 0001:000015e4       Java_jdk_test_lib_jvmti_DebugeeClass_resetAgentData 00000001800025e4 f   libGetStackTraceSuspendedStress.obj
 0001:00001688       __local_stdio_printf_options 0000000180002688 f i libGetStackTraceSuspendedStress.obj
 0001:00001690       agent_resume_sync          0000000180002690 f   libGetStackTraceSuspendedStress.obj
 0001:000017d0       agent_wait_for_sync        00000001800027d0 f   libGetStackTraceSuspendedStress.obj
 0001:00001908       printf                     0000000180002908 f i libGetStackTraceSuspendedStress.obj
 0001:00001e34       _Init_thread_footer        0000000180002e34 f   MSVCRT:thread_safe_statics.obj
 0001:00001e94       _Init_thread_header        0000000180002e94 f   MSVCRT:thread_safe_statics.obj
 0001:00001efc       _Init_thread_notify        0000000180002efc f   MSVCRT:thread_safe_statics.obj
 0001:00001f40       _Init_thread_wait          0000000180002f40 f   MSVCRT:thread_safe_statics.obj
 0001:00001fa4       __GSHandlerCheck           0000000180002fa4 f   MSVCRT:gshandler.obj
 0001:00001fc4       __GSHandlerCheckCommon     0000000180002fc4 f   MSVCRT:gshandler.obj
 0001:00002030       __security_check_cookie    0000000180003030 f   MSVCRT:amdsecgs.obj
 0001:00002370       _DllMainCRTStartup         0000000180003370 f   MSVCRT:dll_dllmain.obj
 0001:000023b0       __scrt_acquire_startup_lock 00000001800033b0 f   MSVCRT:utility.obj
 0001:000023ec       __scrt_dllmain_after_initialize_c 00000001800033ec f   MSVCRT:utility.obj
 0001:00002420       __scrt_dllmain_before_initialize_c 0000000180003420 f   MSVCRT:utility.obj
 0001:00002438       __scrt_dllmain_crt_thread_attach 0000000180003438 f   MSVCRT:utility.obj
 0001:00002460       __scrt_dllmain_crt_thread_detach 0000000180003460 f   MSVCRT:utility.obj
 0001:00002478       __scrt_dllmain_exception_filter 0000000180003478 f   MSVCRT:utility.obj
 0001:000024d8       __scrt_dllmain_uninitialize_c 00000001800034d8 f   MSVCRT:utility.obj
 0001:00002508       __scrt_dllmain_uninitialize_critical 0000000180003508 f   MSVCRT:utility.obj
 0001:0000251c       __scrt_initialize_crt      000000018000351c f   MSVCRT:utility.obj
 0001:00002568       __scrt_initialize_onexit_tables 0000000180003568 f   MSVCRT:utility.obj
 0001:000025f4       __scrt_is_nonwritable_in_current_image 00000001800035f4 f   MSVCRT:utility.obj
 0001:0000268c       __scrt_release_startup_lock 000000018000368c f   MSVCRT:utility.obj
 0001:000026b0       __scrt_uninitialize_crt    00000001800036b0 f   MSVCRT:utility.obj
 0001:000026dc       _onexit                    00000001800036dc f   MSVCRT:utility.obj
 0001:00002718       atexit                     0000000180003718 f   MSVCRT:utility.obj
 0001:00002730       __crt_debugger_hook        0000000180003730 f   MSVCRT:utility_desktop.obj
 0001:00002738       __scrt_fastfail            0000000180003738 f   MSVCRT:utility_desktop.obj
 0001:00002884       _guard_check_icall_nop     0000000180003884 f i MSVCRT:guard_support.obj
 0001:00002888       __raise_securityfailure    0000000180003888 f   MSVCRT:gs_report.obj
 0001:000028bc       __report_gsfailure         00000001800038bc f   MSVCRT:gs_report.obj
 0001:00002a04       __security_init_cookie     0000000180003a04 f   MSVCRT:gs_support.obj
 0001:00002ab0       DllMain                    0000000180003ab0 f   MSVCRT:dll_dllmain_stub.obj
 0001:00002ad4       ?__scrt_initialize_type_info@@YAXXZ 0000000180003ad4 f   MSVCRT:tncleanup.obj
 0001:00002ae4       ?__scrt_uninitialize_type_info@@YAXXZ 0000000180003ae4 f   MSVCRT:tncleanup.obj
 0001:00002af0       __local_stdio_scanf_options 0000000180003af0 f i MSVCRT:default_local_stdio_options.obj
 0001:00002af8       __scrt_initialize_default_local_stdio_options 0000000180003af8 f   MSVCRT:default_local_stdio_options.obj
 0001:00002b14       __scrt_get_dyn_tls_init_callback 0000000180003b14 f   MSVCRT:dyn_tls_init.obj
 0001:00002b1c       _RTC_Initialize            0000000180003b1c f   MSVCRT:initsect.obj
 0001:00002b58       _RTC_Terminate             0000000180003b58 f   MSVCRT:initsect.obj
 0001:00002b94       __isa_available_init       0000000180003b94 f   MSVCRT:cpu_disp.obj
 0001:00002d40       _get_startup_argv_mode     0000000180003d40 f   MSVCRT:argv_mode.obj
 0001:00002d48       __scrt_is_ucrt_dll_in_use  0000000180003d48 f   MSVCRT:ucrt_detection.obj
 0001:00002d60       memset                     0000000180003d60 f   vcruntime:VCRUNTIME140.dll
 0001:00002d66       strstr                     0000000180003d66 f   vcruntime:VCRUNTIME140.dll
 0001:00002d6c       __C_specific_handler       0000000180003d6c f   vcruntime:VCRUNTIME140.dll
 0001:00002d72       __std_type_info_destroy_list 0000000180003d72 f   vcruntime:VCRUNTIME140.dll
 0001:00002d78       strcat                     0000000180003d78 f   ucrt:api-ms-win-crt-string-l1-1-0.dll
 0001:00002d7e       strcmp                     0000000180003d7e f   ucrt:api-ms-win-crt-string-l1-1-0.dll
 0001:00002d84       strlen                     0000000180003d84 f   ucrt:api-ms-win-crt-string-l1-1-0.dll
 0001:00002d8a       _initterm                  0000000180003d8a f   ucrt:api-ms-win-crt-runtime-l1-1-0.dll
 0001:00002d90       _initterm_e                0000000180003d90 f   ucrt:api-ms-win-crt-runtime-l1-1-0.dll
 0001:00002d96       _seh_filter_dll            0000000180003d96 f   ucrt:api-ms-win-crt-runtime-l1-1-0.dll
 0001:00002d9c       _configure_narrow_argv     0000000180003d9c f   ucrt:api-ms-win-crt-runtime-l1-1-0.dll
 0001:00002da2       _initialize_narrow_environment 0000000180003da2 f   ucrt:api-ms-win-crt-runtime-l1-1-0.dll
 0001:00002da8       _initialize_onexit_table   0000000180003da8 f   ucrt:api-ms-win-crt-runtime-l1-1-0.dll
 0001:00002dae       _register_onexit_function  0000000180003dae f   ucrt:api-ms-win-crt-runtime-l1-1-0.dll
 0001:00002db4       _execute_onexit_table      0000000180003db4 f   ucrt:api-ms-win-crt-runtime-l1-1-0.dll
 0001:00002dba       _crt_atexit                0000000180003dba f   ucrt:api-ms-win-crt-runtime-l1-1-0.dll
 0001:00002dc0       _cexit                     0000000180003dc0 f   ucrt:api-ms-win-crt-runtime-l1-1-0.dll
 0001:00002dc8       __acrt_initialize          0000000180003dc8 f   MSVCRT:ucrt_stubs.obj
 0001:00002dc8       __acrt_thread_attach       0000000180003dc8 f   MSVCRT:ucrt_stubs.obj
 0001:00002dc8       __acrt_thread_detach       0000000180003dc8 f   MSVCRT:ucrt_stubs.obj
 0001:00002dc8       __acrt_uninitialize        0000000180003dc8 f   MSVCRT:ucrt_stubs.obj
 0001:00002dc8       __acrt_uninitialize_critical 0000000180003dc8 f   MSVCRT:ucrt_stubs.obj
 0001:00002dc8       __scrt_stub_for_acrt_initialize 0000000180003dc8 f   MSVCRT:ucrt_stubs.obj
 0001:00002dc8       __scrt_stub_for_acrt_thread_attach 0000000180003dc8 f   MSVCRT:ucrt_stubs.obj
 0001:00002dc8       __scrt_stub_for_acrt_thread_detach 0000000180003dc8 f   MSVCRT:ucrt_stubs.obj
 0001:00002dc8       __scrt_stub_for_acrt_uninitialize 0000000180003dc8 f   MSVCRT:ucrt_stubs.obj
 0001:00002dc8       __scrt_stub_for_acrt_uninitialize_critical 0000000180003dc8 f   MSVCRT:ucrt_stubs.obj
 0001:00002dc8       __vcrt_initialize          0000000180003dc8 f   MSVCRT:ucrt_stubs.obj
 0001:00002dc8       __vcrt_thread_attach       0000000180003dc8 f   MSVCRT:ucrt_stubs.obj
 0001:00002dc8       __vcrt_thread_detach       0000000180003dc8 f   MSVCRT:ucrt_stubs.obj
 0001:00002dc8       __vcrt_uninitialize        0000000180003dc8 f   MSVCRT:ucrt_stubs.obj
 0001:00002dc8       __vcrt_uninitialize_critical 0000000180003dc8 f   MSVCRT:ucrt_stubs.obj
 0001:00002dcc       __scrt_stub_for_is_c_termination_complete 0000000180003dcc f   MSVCRT:ucrt_stubs.obj
 0001:00002dcc       _is_c_termination_complete 0000000180003dcc f   MSVCRT:ucrt_stubs.obj
 0001:00002dcf       memcpy                     0000000180003dcf f   vcruntime:VCRUNTIME140.dll
 0001:00002df0       _guard_dispatch_icall_nop  0000000180003df0 f   MSVCRT:guard_dispatch.obj
 0001:00002e10       _guard_xfg_dispatch_icall_nop 0000000180003e10 f   MSVCRT:guard_xfg_dispatch.obj
 0002:00000000       __imp_Sleep                0000000180004000     kernel32:KERNEL32.dll
 0002:00000008       __imp_CloseHandle          0000000180004008     kernel32:KERNEL32.dll
 0002:00000010       __imp_EnterCriticalSection 0000000180004010     kernel32:KERNEL32.dll
 0002:00000018       __imp_LeaveCriticalSection 0000000180004018     kernel32:KERNEL32.dll
 0002:00000020       __imp_InitializeCriticalSectionAndSpinCount 0000000180004020     kernel32:KERNEL32.dll
 0002:00000028       __imp_DeleteCriticalSection 0000000180004028     kernel32:KERNEL32.dll
 0002:00000030       __imp_SetEvent             0000000180004030     kernel32:KERNEL32.dll
 0002:00000038       __imp_ResetEvent           0000000180004038     kernel32:KERNEL32.dll
 0002:00000040       __imp_WaitForSingleObjectEx 0000000180004040     kernel32:KERNEL32.dll
 0002:00000048       __imp_CreateEventW         0000000180004048     kernel32:KERNEL32.dll
 0002:00000050       __imp_GetModuleHandleW     0000000180004050     kernel32:KERNEL32.dll
 0002:00000058       __imp_GetProcAddress       0000000180004058     kernel32:KERNEL32.dll
 0002:00000060       __imp_RtlCaptureContext    0000000180004060     kernel32:KERNEL32.dll
 0002:00000068       __imp_RtlLookupFunctionEntry 0000000180004068     kernel32:KERNEL32.dll
 0002:00000070       __imp_RtlVirtualUnwind     0000000180004070     kernel32:KERNEL32.dll
 0002:00000078       __imp_IsDebuggerPresent    0000000180004078     kernel32:KERNEL32.dll
 0002:00000080       __imp_UnhandledExceptionFilter 0000000180004080     kernel32:KERNEL32.dll
 0002:00000088       __imp_SetUnhandledExceptionFilter 0000000180004088     kernel32:KERNEL32.dll
 0002:00000090       __imp_IsProcessorFeaturePresent 0000000180004090     kernel32:KERNEL32.dll
 0002:00000098       __imp_GetCurrentProcess    0000000180004098     kernel32:KERNEL32.dll
 0002:000000a0       __imp_TerminateProcess     00000001800040a0     kernel32:KERNEL32.dll
 0002:000000a8       __imp_QueryPerformanceCounter 00000001800040a8     kernel32:KERNEL32.dll
 0002:000000b0       __imp_GetCurrentProcessId  00000001800040b0     kernel32:KERNEL32.dll
 0002:000000b8       __imp_GetCurrentThreadId   00000001800040b8     kernel32:KERNEL32.dll
 0002:000000c0       __imp_GetSystemTimeAsFileTime 00000001800040c0     kernel32:KERNEL32.dll
 0002:000000c8       __imp_DisableThreadLibraryCalls 00000001800040c8     kernel32:KERNEL32.dll
 0002:000000d0       __imp_InitializeSListHead  00000001800040d0     kernel32:KERNEL32.dll
 0002:000000d8       \177KERNEL32_NULL_THUNK_DATA 00000001800040d8     kernel32:KERNEL32.dll
 0002:000000e0       __imp_memset               00000001800040e0     vcruntime:VCRUNTIME140.dll
 0002:000000e8       __imp_strstr               00000001800040e8     vcruntime:VCRUNTIME140.dll
 0002:000000f0       __imp___C_specific_handler 00000001800040f0     vcruntime:VCRUNTIME140.dll
 0002:000000f8       __imp___std_type_info_destroy_list 00000001800040f8     vcruntime:VCRUNTIME140.dll
 0002:00000100       __imp_memcpy               0000000180004100     vcruntime:VCRUNTIME140.dll
 0002:00000108       \177VCRUNTIME140_NULL_THUNK_DATA 0000000180004108     vcruntime:VCRUNTIME140.dll
 0002:00000110       __imp__initialize_narrow_environment 0000000180004110     ucrt:api-ms-win-crt-runtime-l1-1-0.dll
 0002:00000118       __imp__cexit               0000000180004118     ucrt:api-ms-win-crt-runtime-l1-1-0.dll
 0002:00000120       __imp__crt_atexit          0000000180004120     ucrt:api-ms-win-crt-runtime-l1-1-0.dll
 0002:00000128       __imp__execute_onexit_table 0000000180004128     ucrt:api-ms-win-crt-runtime-l1-1-0.dll
 0002:00000130       __imp__register_onexit_function 0000000180004130     ucrt:api-ms-win-crt-runtime-l1-1-0.dll
 0002:00000138       __imp__initterm            0000000180004138     ucrt:api-ms-win-crt-runtime-l1-1-0.dll
 0002:00000140       __imp__initterm_e          0000000180004140     ucrt:api-ms-win-crt-runtime-l1-1-0.dll
 0002:00000148       __imp__seh_filter_dll      0000000180004148     ucrt:api-ms-win-crt-runtime-l1-1-0.dll
 0002:00000150       __imp__initialize_onexit_table 0000000180004150     ucrt:api-ms-win-crt-runtime-l1-1-0.dll
 0002:00000158       __imp__configure_narrow_argv 0000000180004158     ucrt:api-ms-win-crt-runtime-l1-1-0.dll
 0002:00000160       \177api-ms-win-crt-runtime-l1-1-0_NULL_THUNK_DATA 0000000180004160     ucrt:api-ms-win-crt-runtime-l1-1-0.dll
 0002:00000168       __imp_fflush               0000000180004168     ucrt:api-ms-win-crt-stdio-l1-1-0.dll
 0002:00000170       __imp___acrt_iob_func      0000000180004170     ucrt:api-ms-win-crt-stdio-l1-1-0.dll
 0002:00000178       __imp___stdio_common_vfprintf 0000000180004178     ucrt:api-ms-win-crt-stdio-l1-1-0.dll
 0002:00000180       \177api-ms-win-crt-stdio-l1-1-0_NULL_THUNK_DATA 0000000180004180     ucrt:api-ms-win-crt-stdio-l1-1-0.dll
 0002:00000188       __imp_strlen               0000000180004188     ucrt:api-ms-win-crt-string-l1-1-0.dll
 0002:00000190       __imp_strncpy              0000000180004190     ucrt:api-ms-win-crt-string-l1-1-0.dll
 0002:00000198       __imp_strcat               0000000180004198     ucrt:api-ms-win-crt-string-l1-1-0.dll
 0002:000001a0       __imp_strcmp               00000001800041a0     ucrt:api-ms-win-crt-string-l1-1-0.dll
 0002:000001a8       \177api-ms-win-crt-string-l1-1-0_NULL_THUNK_DATA 00000001800041a8     ucrt:api-ms-win-crt-string-l1-1-0.dll
 0002:000001b0       __guard_check_icall_fptr   00000001800041b0     MSVCRT:guard_support.obj
 0002:000001b8       __guard_xfg_check_icall_fptr 00000001800041b8     MSVCRT:guard_support.obj
 0002:000001c0       __guard_dispatch_icall_fptr 00000001800041c0     MSVCRT:guard_support.obj
 0002:000001c8       __guard_xfg_dispatch_icall_fptr 00000001800041c8     MSVCRT:guard_support.obj
 0002:000001d0       __guard_xfg_table_dispatch_icall_fptr 00000001800041d0     MSVCRT:guard_support.obj
 0002:000001d8       __castguard_check_failure_os_handled_fptr 00000001800041d8     MSVCRT:guard_support.obj
 0002:000001e0       __guard_memcpy_fptr        00000001800041e0     vcruntime:softmemtag.obj
 0002:000001e8       __xc_a                     00000001800041e8     MSVCRT:initializers.obj
 0002:000001f0       __xc_z                     00000001800041f0     MSVCRT:initializers.obj
 0002:000001f8       __xi_a                     00000001800041f8     MSVCRT:initializers.obj
 0002:00000208       __xi_z                     0000000180004208     MSVCRT:initializers.obj
 0002:00000210       __xl_a                     0000000180004210     MSVCRT:tlssup.obj
 0002:00000218       __xl_z                     0000000180004218     MSVCRT:tlssup.obj
 0002:00000220       __xp_a                     0000000180004220     MSVCRT:initializers.obj
 0002:00000228       __xp_z                     0000000180004228     MSVCRT:initializers.obj
 0002:00000230       __xt_a                     0000000180004230     MSVCRT:initializers.obj
 0002:00000238       __xt_z                     0000000180004238     MSVCRT:initializers.obj
 0002:00000268       ??_C@_0DM@KLJPMIDM@check_jvmti_status?3?5JVMTI?5funct@ 0000000180004268     libGetStackTraceSuspendedStress.obj
 0002:000002a8       ??_C@_0CA@CCEFGCFD@Fatal?5Error?5in?5RawMonitorEnter?4@ 00000001800042a8     libGetStackTraceSuspendedStress.obj
 0002:000002c8       ??_C@_0BP@POHFIHGF@Fatal?5Error?5in?5RawMonitorWait?4@ 00000001800042c8     libGetStackTraceSuspendedStress.obj
 0002:000002e8       ??_C@_0CB@HBCCEOBO@Fatal?5Error?5in?5RawMonitorNotify@ 00000001800042e8     libGetStackTraceSuspendedStress.obj
 0002:00000310       ??_C@_0CL@MEELKAEL@deallocate?3?5error?5in?5JVMTI?5Deal@ 0000000180004310     libGetStackTraceSuspendedStress.obj
 0002:00000340       ??_C@_0DO@CNKPCOHC@get_method_class_name?3?5error?5in@ 0000000180004340     libGetStackTraceSuspendedStress.obj
 0002:00000380       ??_C@_0DI@ODOBMANA@get_method_class_name?3?5error?5in@ 0000000180004380     libGetStackTraceSuspendedStress.obj
 0002:000003b8       ??_C@_0CP@IBPBEBM@get_method_class_name?3?5error?5in@ 00000001800043b8     libGetStackTraceSuspendedStress.obj
 0002:000003e8       ??_C@_0CL@BDMIAND@print_method?3?5error?5in?5JVMTI?5Ge@ 00000001800043e8     libGetStackTraceSuspendedStress.obj
 0002:00000418       ??_C@_0P@GFDDDNG@?$CF2d?3?5?$CFs?3?5?$CFs?$CFs?6@ 0000000180004418     libGetStackTraceSuspendedStress.obj
 0002:00000428       ??_C@_0BH@FJFLJIKN@Error?5in?5GetThreadInfo@ 0000000180004428     libGetStackTraceSuspendedStress.obj
 0002:00000440       ??_C@_06POKJIJFP@daemon@   0000000180004440     libGetStackTraceSuspendedStress.obj
 0002:00000447       ??_C@_00CNPNBAHC@@         0000000180004447     libGetStackTraceSuspendedStress.obj
 0002:00000448       ??_C@_07HIMIIOGA@virtual@  0000000180004448     libGetStackTraceSuspendedStress.obj
 0002:00000450       ??_C@_06GMKELIII@kernel@   0000000180004450     libGetStackTraceSuspendedStress.obj
 0002:00000458       ??_C@_0DD@IEDODGJA@Thread?3?5?$CFp?0?5name?3?5?$CFs?0?5state?$CI?$CFx?$CJ@ 0000000180004458     libGetStackTraceSuspendedStress.obj
 0002:00000490       ??_C@_0CE@NCJONKKC@JVMTI?5Stack?5Trace?3?5frame?5count?3@ 0000000180004490     libGetStackTraceSuspendedStress.obj
 0002:000004b4       ??_C@_01EEMJAFIK@?6@       00000001800044b4     libGetStackTraceSuspendedStress.obj
 0002:000004b8       ??_C@_0DF@MAFJFJPA@get_thread_state?3?5error?5in?5JVMT@ 00000001800044b8     libGetStackTraceSuspendedStress.obj
 0002:000004f0       ??_C@_0BB@NEONAMMP@?$DMUnnamed?5thread?$DO@ 00000001800044f0     libGetStackTraceSuspendedStress.obj
 0002:00000508       ??_C@_0DD@PEIMAGBL@get_thread_name?3?5error?5in?5JVMTI@ 0000000180004508     libGetStackTraceSuspendedStress.obj
 0002:00000540       ??_C@_0DD@GMADJBLO@get_method_name?3?5error?5in?5JVMTI@ 0000000180004540     libGetStackTraceSuspendedStress.obj
 0002:00000578       ??_C@_0DA@DGJBBBMN@print_stack_trace?3?5error?5in?5JVM@ 0000000180004578     libGetStackTraceSuspendedStress.obj
 0002:000005a8       ??_C@_0DC@EJGPEKOE@JVMTI?5Stack?5Trace?5for?5thread?5?$CFs@ 00000001800045a8     libGetStackTraceSuspendedStress.obj
 0002:000005dc       ??_C@_06PAOMPDJH@?$DMnone?$DO@ 00000001800045dc     libGetStackTraceSuspendedStress.obj
 0002:000005e4       ??_C@_06PHAKILGJ@?5ALIVE@  00000001800045e4     libGetStackTraceSuspendedStress.obj
 0002:000005f0       ??_C@_0M@OFKKEJHG@?5TERMINATED@ 00000001800045f0     libGetStackTraceSuspendedStress.obj
 0002:00000600       ??_C@_09JDCMELJI@?5RUNNABLE@ 0000000180004600     libGetStackTraceSuspendedStress.obj
 0002:00000610       ??_C@_08OAHMLBPA@?5WAITING@ 0000000180004610     libGetStackTraceSuspendedStress.obj
 0002:00000620       ??_C@_0BG@GOEBACGE@?5WAITING_INDEFINITELY@ 0000000180004620     libGetStackTraceSuspendedStress.obj
 0002:00000638       ??_C@_0BG@CCLPBKFG@?5WAITING_WITH_TIMEOUT@ 0000000180004638     libGetStackTraceSuspendedStress.obj
 0002:00000650       ??_C@_09DEFAFODN@?5SLEEPING@ 0000000180004650     libGetStackTraceSuspendedStress.obj
 0002:00000660       ??_C@_0BA@EIDDAKGK@?5IN_OBJECT_WAIT@ 0000000180004660     libGetStackTraceSuspendedStress.obj
 0002:00000670       ??_C@_07GIPIPEAD@?5PARKED@ 0000000180004670     libGetStackTraceSuspendedStress.obj
 0002:00000678       ??_C@_0BK@LNIHGEJF@?5BLOCKED_ON_MONITOR_ENTER@ 0000000180004678     libGetStackTraceSuspendedStress.obj
 0002:00000698       ??_C@_0L@MOBKJCJD@?5SUSPENDED@ 0000000180004698     libGetStackTraceSuspendedStress.obj
 0002:000006a8       ??_C@_0N@CPMJCKAP@?5INTERRUPTED@ 00000001800046a8     libGetStackTraceSuspendedStress.obj
 0002:000006b8       ??_C@_0L@PEJNJEEC@?5IN_NATIVE@ 00000001800046b8     libGetStackTraceSuspendedStress.obj
 0002:000006c8       ??_C@_0BB@JCNMKLLK@JVMTI_ERROR_NONE@ 00000001800046c8     libGetStackTraceSuspendedStress.obj
 0002:000006e0       ??_C@_0BL@LDIMKLPH@JVMTI_ERROR_INVALID_THREAD@ 00000001800046e0     libGetStackTraceSuspendedStress.obj
 0002:00000700       ??_C@_0CB@PJFPAIKJ@JVMTI_ERROR_INVALID_THREAD_GROU@ 0000000180004700     libGetStackTraceSuspendedStress.obj
 0002:00000728       ??_C@_0BN@LLMKHMNF@JVMTI_ERROR_INVALID_PRIORITY@ 0000000180004728     libGetStackTraceSuspendedStress.obj
 0002:00000748       ??_C@_0CB@MBOFKAGB@JVMTI_ERROR_THREAD_NOT_SUSPENDE@ 0000000180004748     libGetStackTraceSuspendedStress.obj
 0002:00000770       ??_C@_0BN@FABOLPBI@JVMTI_ERROR_THREAD_SUSPENDED@ 0000000180004770     libGetStackTraceSuspendedStress.obj
 0002:00000790       ??_C@_0BN@FDGNOBJM@JVMTI_ERROR_THREAD_NOT_ALIVE@ 0000000180004790     libGetStackTraceSuspendedStress.obj
 0002:000007b0       ??_C@_0BL@GOBIFKNJ@JVMTI_ERROR_INVALID_OBJECT@ 00000001800047b0     libGetStackTraceSuspendedStress.obj
 0002:000007d0       ??_C@_0BK@FCMAJPPC@JVMTI_ERROR_INVALID_CLASS@ 00000001800047d0     libGetStackTraceSuspendedStress.obj
 0002:000007f0       ??_C@_0BP@IKLLBKEB@JVMTI_ERROR_CLASS_NOT_PREPARED@ 00000001800047f0     libGetStackTraceSuspendedStress.obj
 0002:00000810       ??_C@_0BN@KLPPLKG@JVMTI_ERROR_INVALID_METHODID@ 0000000180004810     libGetStackTraceSuspendedStress.obj
 0002:00000830       ??_C@_0BN@BCEKOKND@JVMTI_ERROR_INVALID_LOCATION@ 0000000180004830     libGetStackTraceSuspendedStress.obj
 0002:00000850       ??_C@_0BM@DFDGPME@JVMTI_ERROR_INVALID_FIELDID@ 0000000180004850     libGetStackTraceSuspendedStress.obj
 0002:00000870       ??_C@_0BL@NELIEPEC@JVMTI_ERROR_NO_MORE_FRAMES@ 0000000180004870     libGetStackTraceSuspendedStress.obj
 0002:00000890       ??_C@_0BJ@BDBECFDM@JVMTI_ERROR_OPAQUE_FRAME@ 0000000180004890     libGetStackTraceSuspendedStress.obj
 0002:000008b0       ??_C@_0BK@MIIFNLOB@JVMTI_ERROR_TYPE_MISMATCH@ 00000001800048b0     libGetStackTraceSuspendedStress.obj
 0002:000008d0       ??_C@_0BJ@HPCAOILC@JVMTI_ERROR_INVALID_SLOT@ 00000001800048d0     libGetStackTraceSuspendedStress.obj
 0002:000008f0       ??_C@_0BG@CHILOPNI@JVMTI_ERROR_DUPLICATE@ 00000001800048f0     libGetStackTraceSuspendedStress.obj
 0002:00000908       ??_C@_0BG@DIEMLHKM@JVMTI_ERROR_NOT_FOUND@ 0000000180004908     libGetStackTraceSuspendedStress.obj
 0002:00000920       ??_C@_0BM@NHMCKHOB@JVMTI_ERROR_INVALID_MONITOR@ 0000000180004920     libGetStackTraceSuspendedStress.obj
 0002:00000940       ??_C@_0BO@PPEDAJGL@JVMTI_ERROR_NOT_MONITOR_OWNER@ 0000000180004940     libGetStackTraceSuspendedStress.obj
 0002:00000960       ??_C@_0BG@FCAIPEID@JVMTI_ERROR_INTERRUPT@ 0000000180004960     libGetStackTraceSuspendedStress.obj
 0002:00000978       ??_C@_0CB@EGDBNKOI@JVMTI_ERROR_INVALID_CLASS_FORMA@ 0000000180004978     libGetStackTraceSuspendedStress.obj
 0002:000009a0       ??_C@_0CG@DGKOGIAL@JVMTI_ERROR_CIRCULAR_CLASS_DEFI@ 00000001800049a0     libGetStackTraceSuspendedStress.obj
 0002:000009c8       ??_C@_0BP@ICEALPKC@JVMTI_ERROR_FAILS_VERIFICATION@ 00000001800049c8     libGetStackTraceSuspendedStress.obj
 0002:000009e8       ??_C@_0DC@JDACLMIO@JVMTI_ERROR_UNSUPPORTED_REDEFIN@ 00000001800049e8     libGetStackTraceSuspendedStress.obj
 0002:00000a20       ??_C@_0DE@GKDKNOMJ@JVMTI_ERROR_UNSUPPORTED_REDEFIN@ 0000000180004a20     libGetStackTraceSuspendedStress.obj
 0002:00000a58       ??_C@_0BO@LAFKIOG@JVMTI_ERROR_INVALID_TYPESTATE@ 0000000180004a58     libGetStackTraceSuspendedStress.obj
 0002:00000a78       ??_C@_0DH@INDGCLLB@JVMTI_ERROR_UNSUPPORTED_REDEFIN@ 0000000180004a78     libGetStackTraceSuspendedStress.obj
 0002:00000ab0       ??_C@_0DE@NHEOMMGI@JVMTI_ERROR_UNSUPPORTED_REDEFIN@ 0000000180004ab0     libGetStackTraceSuspendedStress.obj
 0002:00000ae8       ??_C@_0CA@EKPNJOEP@JVMTI_ERROR_UNSUPPORTED_VERSION@ 0000000180004ae8     libGetStackTraceSuspendedStress.obj
 0002:00000b08       ??_C@_0BN@OFFMAHHL@JVMTI_ERROR_NAMES_DONT_MATCH@ 0000000180004b08     libGetStackTraceSuspendedStress.obj
 0002:00000b28       ??_C@_0DN@HHBBLAKE@JVMTI_ERROR_UNSUPPORTED_REDEFIN@ 0000000180004b28     libGetStackTraceSuspendedStress.obj
 0002:00000b68       ??_C@_0DO@HMBGBGNA@JVMTI_ERROR_UNSUPPORTED_REDEFIN@ 0000000180004b68     libGetStackTraceSuspendedStress.obj
 0002:00000ba8       ??_C@_0BP@PBECGKHJ@JVMTI_ERROR_UNMODIFIABLE_CLASS@ 0000000180004ba8     libGetStackTraceSuspendedStress.obj
 0002:00000bc8       ??_C@_0BK@CANILEHF@JVMTI_ERROR_NOT_AVAILABLE@ 0000000180004bc8     libGetStackTraceSuspendedStress.obj
 0002:00000be8       ??_C@_0CE@INJKMEFK@JVMTI_ERROR_MUST_POSSESS_CAPABI@ 0000000180004be8     libGetStackTraceSuspendedStress.obj
 0002:00000c10       ??_C@_0BJ@LBFPFPDM@JVMTI_ERROR_NULL_POINTER@ 0000000180004c10     libGetStackTraceSuspendedStress.obj
 0002:00000c30       ??_C@_0BP@CHJPNNEM@JVMTI_ERROR_ABSENT_INFORMATION@ 0000000180004c30     libGetStackTraceSuspendedStress.obj
 0002:00000c50       ??_C@_0BP@OMFMNLC@JVMTI_ERROR_INVALID_EVENT_TYPE@ 0000000180004c50     libGetStackTraceSuspendedStress.obj
 0002:00000c70       ??_C@_0BN@BIBNPHHO@JVMTI_ERROR_ILLEGAL_ARGUMENT@ 0000000180004c70     libGetStackTraceSuspendedStress.obj
 0002:00000c90       ??_C@_0BK@KKNDHDCE@JVMTI_ERROR_NATIVE_METHOD@ 0000000180004c90     libGetStackTraceSuspendedStress.obj
 0002:00000cb0       ??_C@_0BK@PMKCFHAE@JVMTI_ERROR_OUT_OF_MEMORY@ 0000000180004cb0     libGetStackTraceSuspendedStress.obj
 0002:00000cd0       ??_C@_0BK@NNJBDMNB@JVMTI_ERROR_ACCESS_DENIED@ 0000000180004cd0     libGetStackTraceSuspendedStress.obj
 0002:00000cf0       ??_C@_0BI@GHECLMNC@JVMTI_ERROR_WRONG_PHASE@ 0000000180004cf0     libGetStackTraceSuspendedStress.obj
 0002:00000d08       ??_C@_0BF@OLIHJOII@JVMTI_ERROR_INTERNAL@ 0000000180004d08     libGetStackTraceSuspendedStress.obj
 0002:00000d20       ??_C@_0BO@EOHGKJHI@JVMTI_ERROR_UNATTACHED_THREAD@ 0000000180004d20     libGetStackTraceSuspendedStress.obj
 0002:00000d40       ??_C@_0CA@LKHFDACL@JVMTI_ERROR_INVALID_ENVIRONMENT@ 0000000180004d40     libGetStackTraceSuspendedStress.obj
 0002:00000d60       ??_C@_0BA@MMFHLOKK@?$DMunknown?5error?$DO@ 0000000180004d60     libGetStackTraceSuspendedStress.obj
 0002:00000d70       ??_C@_0EF@MALILPLA@jvmti_common?5find_ext_function?3@ 0000000180004d70     libGetStackTraceSuspendedStress.obj
 0002:00000db8       ??_C@_0BB@HMLGADFC@GetVirtualThread@ 0000000180004db8     libGetStackTraceSuspendedStress.obj
 0002:00000dd0       ??_C@_0BB@CFFOFLAO@GetCarrierThread@ 0000000180004dd0     libGetStackTraceSuspendedStress.obj
 0002:00000df0       ??_C@_0EL@MEIFBDPD@jvmti_common?5get_virtual_thread@ 0000000180004df0     libGetStackTraceSuspendedStress.obj
 0002:00000e40       ??_C@_0EL@BFBICDJK@jvmti_common?5get_carrier_thread@ 0000000180004e40     libGetStackTraceSuspendedStress.obj
 0002:00000e90       ??_C@_0BD@HGNAOMCP@agent_data_monitor@ 0000000180004e90     libGetStackTraceSuspendedStress.obj
 0002:00000ea8       ??_C@_0CO@PGPGMHBJ@No?5status?5sync?5occured?5for?5time@ 0000000180004ea8     libGetStackTraceSuspendedStress.obj
 0002:00000ed8       ??_C@_0CL@DOEBDPKJ@Debuggee?5was?5not?5suspended?5on?5s@ 0000000180004ed8     libGetStackTraceSuspendedStress.obj
 0002:00000f08       ??_C@_0BD@KDBALNLB@JVMTI?5agent?5thread@ 0000000180004f08     libGetStackTraceSuspendedStress.obj
 0002:00000f20       ??_C@_0BB@NOKBFPFO@java?1lang?1Thread@ 0000000180004f20     libGetStackTraceSuspendedStress.obj
 0002:00000f34       ??_C@_06FALKBLGB@?$DMinit?$DO@ 0000000180004f34     libGetStackTraceSuspendedStress.obj
 0002:00000f40       ??_C@_0BG@IKDDPPGD@?$CILjava?1lang?1String?$DL?$CJV@ 0000000180004f40     libGetStackTraceSuspendedStress.obj
 0002:00000f58       ??_C@_0M@FENMFJM@Data?5?$CFp?5?$CFp?6@ 0000000180004f58     libGetStackTraceSuspendedStress.obj
 0002:00000f70       ??_C@_0EA@MOJDNKDF@Debuggee?5status?5sync?5aborted?5be@ 0000000180004f70     libGetStackTraceSuspendedStress.obj
 0002:00000fb0       ??_C@_0BE@FADCDGEH@FAIL?3?5Status?5is?5?$CFd?6@ 0000000180004fb0     libGetStackTraceSuspendedStress.obj
 0002:00000fc8       ??_C@_0CP@ECJCJOLE@Synchronization?5point?5checkStat@ 0000000180004fc8     libGetStackTraceSuspendedStress.obj
 0002:00000ff8       ??_C@_0BH@MMGMHADI@Error?5in?5GetStackTrace@ 0000000180004ff8     libGetStackTraceSuspendedStress.obj
 0002:00001010       ??_C@_0CM@BCCFPJGJ@Stacktrace?5in?5virtual?5thread?5is@ 0000000180005010     libGetStackTraceSuspendedStress.obj
 0002:00001040       ??_C@_0BK@ONKLMCGF@Incorrect?5frame?5count?5?$CFd?6@ 0000000180005040     libGetStackTraceSuspendedStress.obj
 0002:00001060       ??_C@_0CC@IJFNGPJA@Incorrect?5frame?5count?3?5count?5?$DM?$DN@ 0000000180005060     libGetStackTraceSuspendedStress.obj
 0002:00001090       ??_C@_0EL@FJIKHJNF@Stacktrace?5in?5virtual?5thread?5is@ 0000000180005090     libGetStackTraceSuspendedStress.obj
 0002:000010e0       ??_C@_0BG@NCJEIDAK@incorrect?5stacktrace?4@ 00000001800050e0     libGetStackTraceSuspendedStress.obj
 0002:000010f8       ??_C@_0BH@FJLPBAAC@Error?5in?5GetFrameCount@ 00000001800050f8     libGetStackTraceSuspendedStress.obj
 0002:00001110       ??_C@_0CM@FPAOJEOF@Incorrect?5frame?5count?5?$CFd?5while?5@ 0000000180005110     libGetStackTraceSuspendedStress.obj
 0002:00001140       ??_C@_0CE@OPLIDPME@Suspended?5vthread?51st?5stack?5tra@ 0000000180005140     libGetStackTraceSuspendedStress.obj
 0002:00001168       ??_C@_0CE@OGPGOGFH@Suspended?5vthread?52nd?5stack?5tra@ 0000000180005168     libGetStackTraceSuspendedStress.obj
 0002:00001190       ??_C@_0CM@MDIELBBA@Incorrect?5frame?5count?3?5frame_co@ 0000000180005190     libGetStackTraceSuspendedStress.obj
 0002:000011c0       ??_C@_0CL@CLEEMOPG@Virtual?5thread?5IS?5expected?5to?5b@ 00000001800051c0     libGetStackTraceSuspendedStress.obj
 0002:000011f0       ??_C@_0CP@DNKMEJLI@Carrier?5thread?5is?5NOT?5expected?5@ 00000001800051f0     libGetStackTraceSuspendedStress.obj
 0002:00001220       ??_C@_0L@NOKHOCGA@?6Carrier?3?5@ 0000000180005220     libGetStackTraceSuspendedStress.obj
 0002:00001230       ??_C@_0L@MNFCJGPK@Expected?3?5@ 0000000180005230     libGetStackTraceSuspendedStress.obj
 0002:00001240       ??_C@_0L@CLLBDAON@Resulted?3?5@ 0000000180005240     libGetStackTraceSuspendedStress.obj
 0002:00001250       ??_C@_0DH@LEMCHCJC@GetVirtualThread?$CIGetCarrierThre@ 0000000180005250     libGetStackTraceSuspendedStress.obj
 0002:00001290       ??_C@_0EO@IODAIB@Agent?3?5check_vthread_consistenc@ 0000000180005290     libGetStackTraceSuspendedStress.obj
 0002:000012e0       ??_C@_0DM@LJAEPNIM@Error?5in?5JVMTI?5SetEventNotifica@ 00000001800052e0     libGetStackTraceSuspendedStress.obj
 0002:00001320       ??_C@_0DN@MHHDBCAK@Error?5in?5JVMTI?5SetEventNotifica@ 0000000180005320     libGetStackTraceSuspendedStress.obj
 0002:00001360       ??_C@_0BO@JKAMHDIO@Agent?3?5Got?5SingleStep?5event?3?6@ 0000000180005360     libGetStackTraceSuspendedStress.obj
 0002:00001380       ??_C@_0CB@DLANBIJF@SingleStep?5event?5is?5NOT?5expecte@ 0000000180005380     libGetStackTraceSuspendedStress.obj
 0002:000013a8       ??_C@_0BJ@PJOBAJEC@Agent?3?5waiting?5to?5start?6@ 00000001800053a8     libGetStackTraceSuspendedStress.obj
 0002:000013c8       ??_C@_0BA@CLFGEFPI@Agent?3?5started?6@ 00000001800053c8     libGetStackTraceSuspendedStress.obj
 0002:000013d8       ??_C@_0BH@FLMCGFGL@Error?5in?5GetAllThreads@ 00000001800053d8     libGetStackTraceSuspendedStress.obj
 0002:000013f0       ??_C@_0BK@PIFAIIBC@Error?5in?5GetVirtualThread@ 00000001800053f0     libGetStackTraceSuspendedStress.obj
 0002:00001410       ??_C@_0BH@MJONCJMH@Error?5in?5SuspendThread@ 0000000180005410     libGetStackTraceSuspendedStress.obj
 0002:00001428       ??_C@_0BG@DMPIHLFJ@Error?5in?5ResumeThread@ 0000000180005428     libGetStackTraceSuspendedStress.obj
 0002:00001440       ??_C@_0BE@LLJICBPG@Error?5in?5Deallocate@ 0000000180005440     libGetStackTraceSuspendedStress.obj
 0002:00001458       ??_C@_0BG@FLGBOFJG@Agent_OnLoad?5started?6@ 0000000180005458     libGetStackTraceSuspendedStress.obj
 0002:00001470       ??_C@_0CE@FKKGLAHF@error?5in?5JVMTI?5AddCapabilities?3@ 0000000180005470     libGetStackTraceSuspendedStress.obj
 0002:00001498       ??_C@_0DE@CPNIEIDP@Agent_OnLoad?3?5Error?5in?5JVMTI?5Se@ 0000000180005498     libGetStackTraceSuspendedStress.obj
 0002:000014d0       ??_C@_0P@BDFDLKIL@Events?5Monitor@ 00000001800054d0     libGetStackTraceSuspendedStress.obj
 0002:000014e0       ??_C@_0BH@NMEJPPEK@Agent_OnLoad?5finished?6@ 00000001800054e0     libGetStackTraceSuspendedStress.obj
 0002:00001500       ??_C@_1EC@JIJBPKFM@?$AAa?$AAp?$AAi?$AA?9?$AAm?$AAs?$AA?9?$AAw?$AAi?$AAn?$AA?9?$AAc?$AAo?$AAr?$AAe@ 0000000180005500     MSVCRT:thread_safe_statics.obj
 0002:00001548       ??_C@_1BK@MGMFAEKH@?$AAk?$AAe?$AAr?$AAn?$AAe?$AAl?$AA3?$AA2?$AA?4?$AAd?$AAl?$AAl@ 0000000180005548     MSVCRT:thread_safe_statics.obj
 0002:00001568       ??_C@_0BJ@JEBJOJFJ@SleepConditionVariableCS@ 0000000180005568     MSVCRT:thread_safe_statics.obj
 0002:00001588       ??_C@_0BJ@PGPPEPCC@WakeAllConditionVariable@ 0000000180005588     MSVCRT:thread_safe_statics.obj
 0002:000015a8       _pDefaultRawDllMain        00000001800055a8     MSVCRT:dll_dllmain.obj
 0002:000015a8       _pRawDllMain               00000001800055a8     MSVCRT:dll_dllmain.obj
 0002:000015b0       __xmm@ffffffffffffffffffffffffffffffff 00000001800055b0     MSVCRT:utility.obj
 0002:000015d0       _load_config_used          00000001800055d0     MSVCRT:loadcfg.obj
 0002:00001780       _tls_used                  0000000180005780     MSVCRT:tlssup.obj
 0002:000017a8       __volatile_metadata        00000001800057a8     <linker-defined>
 0002:00001b90       __rtc_iaa                  0000000180005b90     MSVCRT:initsect.obj
 0002:00001b98       __rtc_izz                  0000000180005b98     MSVCRT:initsect.obj
 0002:00001ba0       __rtc_taa                  0000000180005ba0     MSVCRT:initsect.obj
 0002:00001ba8       __rtc_tzz                  0000000180005ba8     MSVCRT:initsect.obj
 0002:00001bb0       _tls_start                 0000000180005bb0     MSVCRT:tlssup.obj
 0002:00001bb4       _Init_thread_epoch         0000000180005bb4     MSVCRT:thread_safe_statics.obj
 0002:00001bb8       _tls_end                   0000000180005bb8     MSVCRT:tlssup.obj
 0002:00001f7c       __IMPORT_DESCRIPTOR_KERNEL32 0000000180005f7c     kernel32:KERNEL32.dll
 0002:00001f90       __IMPORT_DESCRIPTOR_VCRUNTIME140 0000000180005f90     vcruntime:VCRUNTIME140.dll
 0002:00001fa4       __IMPORT_DESCRIPTOR_api-ms-win-crt-string-l1-1-0 0000000180005fa4     ucrt:api-ms-win-crt-string-l1-1-0.dll
 0002:00001fb8       __IMPORT_DESCRIPTOR_api-ms-win-crt-stdio-l1-1-0 0000000180005fb8     ucrt:api-ms-win-crt-stdio-l1-1-0.dll
 0002:00001fcc       __IMPORT_DESCRIPTOR_api-ms-win-crt-runtime-l1-1-0 0000000180005fcc     ucrt:api-ms-win-crt-runtime-l1-1-0.dll
 0002:00001fe0       __NULL_IMPORT_DESCRIPTOR   0000000180005fe0     kernel32:KERNEL32.dll
 0003:00000008       _Init_global_epoch         0000000180007008     MSVCRT:thread_safe_statics.obj
 0003:00000010       __security_cookie          0000000180007010     MSVCRT:gs_cookie.obj
 0003:00000018       __security_cookie_complement 0000000180007018     MSVCRT:gs_cookie.obj
 0003:00000020       __scrt_native_dllmain_reason 0000000180007020     MSVCRT:utility.obj
 0003:00000028       __isa_available            0000000180007028     MSVCRT:cpu_disp.obj
 0003:0000002c       __isa_enabled              000000018000702c     MSVCRT:cpu_disp.obj
 0003:00000030       __memset_fast_string_threshold 0000000180007030     MSVCRT:cpu_disp.obj
 0003:00000038       __memset_nt_threshold      0000000180007038     MSVCRT:cpu_disp.obj
 0003:00000040       __scrt_ucrt_dll_is_in_use  0000000180007040     MSVCRT:ucrt_stubs.obj
 0003:00000050       ?_OptionsStorage@?1??__local_stdio_printf_options@@9@4_KA 0000000180007050     libGetStackTraceSuspendedStress.obj
 0003:00000240       _tls_index                 0000000180007240     MSVCRT:tlssup.obj
 0003:00000248       __scrt_current_native_startup_state 0000000180007248     MSVCRT:utility.obj
 0003:00000250       __scrt_native_startup_lock 0000000180007250     MSVCRT:utility.obj
 0003:00000290       __scrt_debugger_hook_flag  0000000180007290     MSVCRT:utility_desktop.obj
 0003:00000810       ?__type_info_root_node@@3U__type_info_node@@A 0000000180007810     MSVCRT:tncleanup.obj
 0003:00000820       ?_OptionsStorage@?1??__local_stdio_scanf_options@@9@4_KA 0000000180007820     MSVCRT:default_local_stdio_options.obj
 0003:00000828       __favor                    0000000180007828     MSVCRT:cpu_disp.obj
 0003:00000830       __dyn_tls_init_callback    0000000180007830     <common>

 entry point at        0001:00002370

 Static symbols

 0000:ffff6000       .debug$S                   0000000180000000     GetStackTraceSuspendedStress.exp
 0000:ffff6000       .debug$S                   0000000180000000     vcruntime:VCRUNTIME140.dll
 0000:ffff6000       .debug$S                   0000000180000000     vcruntime:VCRUNTIME140.dll
 0000:ffff6000       .debug$S                   0000000180000000     vcruntime:VCRUNTIME140.dll
 0000:ffff6000       .debug$S                   0000000180000000     vcruntime:VCRUNTIME140.dll
 0000:ffff6000       .debug$S                   0000000180000000     vcruntime:VCRUNTIME140.dll
 0000:ffff6000       .debug$S                   0000000180000000     vcruntime:VCRUNTIME140.dll
 0000:ffff6000       .debug$S                   0000000180000000     vcruntime:VCRUNTIME140.dll
 0000:ffff6000       .debug$S                   0000000180000000     ucrt:api-ms-win-crt-runtime-l1-1-0.dll
 0000:ffff6000       .debug$S                   0000000180000000     ucrt:api-ms-win-crt-runtime-l1-1-0.dll
 0000:ffff6000       .debug$S                   0000000180000000     ucrt:api-ms-win-crt-runtime-l1-1-0.dll
 0000:ffff6000       .debug$S                   0000000180000000     ucrt:api-ms-win-crt-runtime-l1-1-0.dll
 0000:ffff6000       .debug$S                   0000000180000000     ucrt:api-ms-win-crt-runtime-l1-1-0.dll
 0000:ffff6000       .debug$S                   0000000180000000     ucrt:api-ms-win-crt-runtime-l1-1-0.dll
 0000:ffff6000       .debug$S                   0000000180000000     ucrt:api-ms-win-crt-runtime-l1-1-0.dll
 0000:ffff6000       .debug$S                   0000000180000000     ucrt:api-ms-win-crt-runtime-l1-1-0.dll
 0000:ffff6000       .debug$S                   0000000180000000     ucrt:api-ms-win-crt-runtime-l1-1-0.dll
 0000:ffff6000       .debug$S                   0000000180000000     ucrt:api-ms-win-crt-runtime-l1-1-0.dll
 0000:ffff6000       .debug$S                   0000000180000000     ucrt:api-ms-win-crt-runtime-l1-1-0.dll
 0000:ffff6000       .debug$S                   0000000180000000     ucrt:api-ms-win-crt-runtime-l1-1-0.dll
 0000:ffff6000       .debug$S                   0000000180000000     ucrt:api-ms-win-crt-runtime-l1-1-0.dll
 0000:ffff6000       .debug$S                   0000000180000000     ucrt:api-ms-win-crt-stdio-l1-1-0.dll
 0000:ffff6000       .debug$S                   0000000180000000     ucrt:api-ms-win-crt-stdio-l1-1-0.dll
 0000:ffff6000       .debug$S                   0000000180000000     ucrt:api-ms-win-crt-stdio-l1-1-0.dll
 0000:ffff6000       .debug$S                   0000000180000000     ucrt:api-ms-win-crt-string-l1-1-0.dll
 0000:ffff6000       .debug$S                   0000000180000000     ucrt:api-ms-win-crt-string-l1-1-0.dll
 0000:ffff6000       .debug$S                   0000000180000000     ucrt:api-ms-win-crt-string-l1-1-0.dll
 0000:ffff6000       .debug$S                   0000000180000000     ucrt:api-ms-win-crt-string-l1-1-0.dll
 0000:ffff6000       .debug$S                   0000000180000000     ucrt:api-ms-win-crt-string-l1-1-0.dll
 0000:ffff6000       .debug$S                   0000000180000000     kernel32:KERNEL32.dll
 0000:ffff6000       .debug$S                   0000000180000000     kernel32:KERNEL32.dll
 0000:ffff6000       .debug$S                   0000000180000000     kernel32:KERNEL32.dll
 0000:ffff6000       .debug$S                   0000000180000000     kernel32:KERNEL32.dll
 0000:ffff6000       .debug$S                   0000000180000000     kernel32:KERNEL32.dll
 0000:ffff6000       .debug$S                   0000000180000000     kernel32:KERNEL32.dll
 0000:ffff6000       .debug$S                   0000000180000000     kernel32:KERNEL32.dll
 0000:ffff6000       .debug$S                   0000000180000000     kernel32:KERNEL32.dll
 0000:ffff6000       .debug$S                   0000000180000000     kernel32:KERNEL32.dll
 0000:ffff6000       .debug$S                   0000000180000000     kernel32:KERNEL32.dll
 0000:ffff6000       .debug$S                   0000000180000000     kernel32:KERNEL32.dll
 0000:ffff6000       .debug$S                   0000000180000000     kernel32:KERNEL32.dll
 0000:ffff6000       .debug$S                   0000000180000000     kernel32:KERNEL32.dll
 0000:ffff6000       .debug$S                   0000000180000000     kernel32:KERNEL32.dll
 0000:ffff6000       .debug$S                   0000000180000000     kernel32:KERNEL32.dll
 0000:ffff6000       .debug$S                   0000000180000000     kernel32:KERNEL32.dll
 0000:ffff6000       .debug$S                   0000000180000000     kernel32:KERNEL32.dll
 0000:ffff6000       .debug$S                   0000000180000000     kernel32:KERNEL32.dll
 0000:ffff6000       .debug$S                   0000000180000000     kernel32:KERNEL32.dll
 0000:ffff6000       .debug$S                   0000000180000000     kernel32:KERNEL32.dll
 0000:ffff6000       .debug$S                   0000000180000000     kernel32:KERNEL32.dll
 0000:ffff6000       .debug$S                   0000000180000000     kernel32:KERNEL32.dll
 0000:ffff6000       .debug$S                   0000000180000000     kernel32:KERNEL32.dll
 0000:ffff6000       .debug$S                   0000000180000000     kernel32:KERNEL32.dll
 0000:ffff6000       .debug$S                   0000000180000000     kernel32:KERNEL32.dll
 0000:ffff6000       .debug$S                   0000000180000000     kernel32:KERNEL32.dll
 0000:ffff6000       .debug$S                   0000000180000000     kernel32:KERNEL32.dll
 0000:ffff6000       .debug$S                   0000000180000000     kernel32:KERNEL32.dll
 0001:0000002c       ?SingleStep@@YAXPEAU_jvmtiEnv@@PEAUJNIEnv_@@PEAV_jobject@@PEAU_jmethodID@@_J@Z 000000018000102c f   libGetStackTraceSuspendedStress.obj
 0001:00000514       ?agentProc@@YAXPEAU_jvmtiEnv@@PEAUJNIEnv_@@PEAX@Z 0000000180001514 f   libGetStackTraceSuspendedStress.obj
 0001:000006f8       ?check_jvmti_status@@YAXPEAUJNIEnv_@@W4jvmtiError@@PEBD@Z 00000001800016f8 f   libGetStackTraceSuspendedStress.obj
 0001:0000096c       ?check_vthread_consistency_suspended@@YAXPEAU_jvmtiEnv@@PEAUJNIEnv_@@PEAV_jobject@@@Z 000000018000196c f   libGetStackTraceSuspendedStress.obj
 0001:00000a3c       ?find_ext_function@@YAP6A?AW4jvmtiError@@PEAU_jvmtiEnv@@ZZ0PEAUJNIEnv_@@PEBD@Z 0000000180001a3c f   libGetStackTraceSuspendedStress.obj
 0001:00000ad0       ?get_carrier_thread@@YAPEAV_jobject@@PEAU_jvmtiEnv@@PEAUJNIEnv_@@PEAV1@@Z 0000000180001ad0 f   libGetStackTraceSuspendedStress.obj
 0001:00000b40       ?get_method_class_name@@YAPEADPEAU_jvmtiEnv@@PEAUJNIEnv_@@PEAU_jmethodID@@@Z 0000000180001b40 f   libGetStackTraceSuspendedStress.obj
 0001:00000c34       ?print_method@@YAXPEAU_jvmtiEnv@@PEAUJNIEnv_@@PEAU_jmethodID@@H@Z 0000000180001c34 f   libGetStackTraceSuspendedStress.obj
 0001:00000d44       ?print_stack_trace@@YAXPEAU_jvmtiEnv@@PEAUJNIEnv_@@PEAV_jobject@@@Z 0000000180001d44 f   libGetStackTraceSuspendedStress.obj
 0001:00000f88       ?print_stack_trace_frames@@YAXPEAU_jvmtiEnv@@PEAUJNIEnv_@@HPEAUjvmtiFrameInfo@@@Z 0000000180001f88 f   libGetStackTraceSuspendedStress.obj
 0001:00001124       ?test_stack_trace@@YAXPEAU_jvmtiEnv@@PEAUJNIEnv_@@PEAV_jobject@@@Z 0000000180002124 f   libGetStackTraceSuspendedStress.obj
 0001:0000176c       agent_thread_wrapper       000000018000276c f   libGetStackTraceSuspendedStress.obj
 0001:0000195c       run_agent_thread           000000018000295c f   libGetStackTraceSuspendedStress.obj
 0001:00001a9c       set_agent_thread_state     0000000180002a9c f   libGetStackTraceSuspendedStress.obj
 0001:00001b44       sync_debuggee_status       0000000180002b44 f   libGetStackTraceSuspendedStress.obj
 0001:00001d3c       ?__scrt_initialize_thread_safe_statics@@YAHXZ 0000000180002d3c f   MSVCRT:thread_safe_statics.obj
 0001:00001e0c       ?__scrt_uninitialize_thread_safe_statics@@YAXXZ 0000000180002e0c f   MSVCRT:thread_safe_statics.obj
 0001:00002020       $$000000                   0000000180003020     MSVCRT:amdsecgs.obj
 0001:00002050       ?dllmain_crt_dispatch@@YAHQEAUHINSTANCE__@@KQEAX@Z 0000000180003050 f   MSVCRT:dll_dllmain.obj
 0001:000020a0       ?dllmain_crt_process_attach@@YAHQEAUHINSTANCE__@@QEAX@Z 00000001800030a0 f   MSVCRT:dll_dllmain.obj
 0001:000021b8       ?dllmain_crt_process_detach@@YAH_N@Z 00000001800031b8 f   MSVCRT:dll_dllmain.obj
 0001:0000223c       ?dllmain_dispatch@@YAHQEAUHINSTANCE__@@KQEAX@Z 000000018000323c f   MSVCRT:dll_dllmain.obj
 0001:00002990       capture_previous_context   0000000180003990 f   MSVCRT:gs_report.obj
 0001:00002de0       $$000000                   0000000180003de0     MSVCRT:guard_dispatch.obj
 0001:00002e00       $$000000                   0000000180003e00     MSVCRT:guard_xfg_dispatch.obj
 0001:00002e16       ?fin$0@?0??dllmain_crt_process_attach@@YAHQEAUHINSTANCE__@@QEAX@Z@4HA 0000000180003e16 f   MSVCRT:dll_dllmain.obj
 0001:00002e2d       ?fin$0@?0??dllmain_crt_process_detach@@YAH_N@Z@4HA 0000000180003e2d f   MSVCRT:dll_dllmain.obj
 0001:00002e46       ?fin$1@?0??dllmain_crt_process_detach@@YAH_N@Z@4HA 0000000180003e46 f   MSVCRT:dll_dllmain.obj
 0001:00002e5a       ?filt$0@?0??dllmain_dispatch@@YAHQEAUHINSTANCE__@@KQEAX@Z@4HA 0000000180003e5a f   MSVCRT:dll_dllmain.obj
 0001:00002e90       __scrt_is_nonwritable_in_current_image$filt$0 0000000180003e90 f   MSVCRT:utility.obj
 0002:00000200       ?__scrt_initialize_tss_var@@3P6AHXZEA 0000000180004200     MSVCRT:thread_safe_statics.obj
 0002:00000240       ?CONTINUATION_CLASS_NAME@@3QBDB 0000000180004240     libGetStackTraceSuspendedStress.obj
 0002:00000260       ?CONTINUATION_METHOD_NAME@@3QBDB 0000000180004260     libGetStackTraceSuspendedStress.obj
 0002:000015c0       GS_ExceptionPointers       00000001800055c0     MSVCRT:gs_report.obj
 0002:00001bc0       $unwind$printf             0000000180005bc0     libGetStackTraceSuspendedStress.obj
 0002:00001bcc       $unwind$?NewObject@JNIEnv_@@QEAAPEAV_jobject@@PEAV_jclass@@PEAU_jmethodID@@ZZ 0000000180005bcc     libGetStackTraceSuspendedStress.obj
 0002:00001bd4       $unwind$Agent_OnLoad       0000000180005bd4     libGetStackTraceSuspendedStress.obj
 0002:00001bf0       $unwind$?TranslateState@@YAPEBDH@Z 0000000180005bf0     libGetStackTraceSuspendedStress.obj
 0002:00001bf0       $unwind$Java_jdk_test_lib_jvmti_DebugeeClass_checkStatus 0000000180005bf0     libGetStackTraceSuspendedStress.obj
 0002:00001bf0       $unwind$agent_thread_wrapper 0000000180005bf0     libGetStackTraceSuspendedStress.obj
 0002:00001bf0       $unwind$_RTC_Initialize    0000000180005bf0     MSVCRT:initsect.obj
 0002:00001bf0       $unwind$_RTC_Terminate     0000000180005bf0     MSVCRT:initsect.obj
 0002:00001bf0       $unwind$?__scrt_initialize_thread_safe_statics@@YAHXZ 0000000180005bf0     MSVCRT:thread_safe_statics.obj
 0002:00001bfc       $unwind$?check_jvmti_status@@YAXPEAUJNIEnv_@@W4jvmtiError@@PEBD@Z 0000000180005bfc     libGetStackTraceSuspendedStress.obj
 0002:00001c0c       $unwind$?get_method_class_name@@YAPEADPEAU_jvmtiEnv@@PEAUJNIEnv_@@PEAU_jmethodID@@@Z 0000000180005c0c     libGetStackTraceSuspendedStress.obj
 0002:00001c1c       $unwind$?print_method@@YAXPEAU_jvmtiEnv@@PEAUJNIEnv_@@PEAU_jmethodID@@H@Z 0000000180005c1c     libGetStackTraceSuspendedStress.obj
 0002:00001c30       $unwind$?print_thread_info@@YAXPEAU_jvmtiEnv@@PEAUJNIEnv_@@PEAV_jobject@@@Z 0000000180005c30     libGetStackTraceSuspendedStress.obj
 0002:00001c40       $unwind$?print_stack_trace_frames@@YAXPEAU_jvmtiEnv@@PEAUJNIEnv_@@HPEAUjvmtiFrameInfo@@@Z 0000000180005c40     libGetStackTraceSuspendedStress.obj
 0002:00001c58       $unwind$?print_stack_trace@@YAXPEAU_jvmtiEnv@@PEAUJNIEnv_@@PEAV_jobject@@@Z 0000000180005c58     libGetStackTraceSuspendedStress.obj
 0002:00001c78       $unwind$?find_ext_function@@YAP6A?AW4jvmtiError@@PEAU_jvmtiEnv@@ZZ0PEAUJNIEnv_@@PEBD@Z 0000000180005c78     libGetStackTraceSuspendedStress.obj
 0002:00001c88       $unwind$?get_carrier_thread@@YAPEAV_jobject@@PEAU_jvmtiEnv@@PEAUJNIEnv_@@PEAV1@@Z 0000000180005c88     libGetStackTraceSuspendedStress.obj
 0002:00001c88       $unwind$Java_jdk_test_lib_jvmti_DebugeeClass_resetAgentData 0000000180005c88     libGetStackTraceSuspendedStress.obj
 0002:00001c88       $unwind$agent_resume_sync  0000000180005c88     libGetStackTraceSuspendedStress.obj
 0002:00001c88       $unwind$_DllMainCRTStartup 0000000180005c88     MSVCRT:dll_dllmain.obj
 0002:00001c98       $unwind$agent_wait_for_sync 0000000180005c98     libGetStackTraceSuspendedStress.obj
 0002:00001cb0       $unwind$?SingleStep@@YAXPEAU_jvmtiEnv@@PEAUJNIEnv_@@PEAV_jobject@@PEAU_jmethodID@@_J@Z 0000000180005cb0     libGetStackTraceSuspendedStress.obj
 0002:00001cb0       $unwind$?check_vthread_consistency_suspended@@YAXPEAU_jvmtiEnv@@PEAUJNIEnv_@@PEAV_jobject@@@Z 0000000180005cb0     libGetStackTraceSuspendedStress.obj
 0002:00001cb0       $unwind$set_agent_thread_state 0000000180005cb0     libGetStackTraceSuspendedStress.obj
 0002:00001cb0       $unwind$__scrt_dllmain_exception_filter 0000000180005cb0     MSVCRT:utility.obj
 0002:00001cc4       $unwind$run_agent_thread   0000000180005cc4     libGetStackTraceSuspendedStress.obj
 0002:00001cd8       $unwind$sync_debuggee_status 0000000180005cd8     libGetStackTraceSuspendedStress.obj
 0002:00001cf4       $unwind$?test_stack_trace@@YAXPEAU_jvmtiEnv@@PEAUJNIEnv_@@PEAV_jobject@@@Z 0000000180005cf4     libGetStackTraceSuspendedStress.obj
 0002:00001d14       $unwind$?check_link_consistency@@YAXPEAU_jvmtiEnv@@PEAUJNIEnv_@@PEAV_jobject@@@Z 0000000180005d14     libGetStackTraceSuspendedStress.obj
 0002:00001d28       $unwind$?agentProc@@YAXPEAU_jvmtiEnv@@PEAUJNIEnv_@@PEAX@Z 0000000180005d28     libGetStackTraceSuspendedStress.obj
 0002:00001d40       $unwind$__raise_securityfailure 0000000180005d40     MSVCRT:gs_report.obj
 0002:00001d40       $unwind$_Init_thread_footer 0000000180005d40     MSVCRT:thread_safe_statics.obj
 0002:00001d40       $unwind$_Init_thread_header 0000000180005d40     MSVCRT:thread_safe_statics.obj
 0002:00001d40       $unwind$_Init_thread_wait  0000000180005d40     MSVCRT:thread_safe_statics.obj
 0002:00001d40       $unwind$__scrt_initialize_crt 0000000180005d40     MSVCRT:utility.obj
 0002:00001d40       $unwind$__scrt_initialize_onexit_tables 0000000180005d40     MSVCRT:utility.obj
 0002:00001d40       $unwind$__scrt_release_startup_lock 0000000180005d40     MSVCRT:utility.obj
 0002:00001d40       $unwind$__scrt_uninitialize_crt 0000000180005d40     MSVCRT:utility.obj
 0002:00001d40       $unwind$_onexit            0000000180005d40     MSVCRT:utility.obj
 0002:00001d48       $unwind$__scrt_initialize_default_local_stdio_options 0000000180005d48     MSVCRT:default_local_stdio_options.obj
 0002:00001d48       $unwind$?dllmain_crt_dispatch@@YAHQEAUHINSTANCE__@@KQEAX@Z 0000000180005d48     MSVCRT:dll_dllmain.obj
 0002:00001d48       $unwind$DllMain            0000000180005d48     MSVCRT:dll_dllmain_stub.obj
 0002:00001d48       $unwind$__GSHandlerCheck   0000000180005d48     MSVCRT:gshandler.obj
 0002:00001d48       $unwind$?__scrt_uninitialize_thread_safe_statics@@YAXXZ 0000000180005d48     MSVCRT:thread_safe_statics.obj
 0002:00001d48       $unwind$_Init_thread_notify 0000000180005d48     MSVCRT:thread_safe_statics.obj
 0002:00001d48       $unwind$__scrt_acquire_startup_lock 0000000180005d48     MSVCRT:utility.obj
 0002:00001d48       $unwind$__scrt_dllmain_after_initialize_c 0000000180005d48     MSVCRT:utility.obj
 0002:00001d48       $unwind$__scrt_dllmain_before_initialize_c 0000000180005d48     MSVCRT:utility.obj
 0002:00001d48       $unwind$__scrt_dllmain_crt_thread_attach 0000000180005d48     MSVCRT:utility.obj
 0002:00001d48       $unwind$__scrt_dllmain_crt_thread_detach 0000000180005d48     MSVCRT:utility.obj
 0002:00001d48       $unwind$__scrt_dllmain_uninitialize_c 0000000180005d48     MSVCRT:utility.obj
 0002:00001d48       $unwind$__scrt_dllmain_uninitialize_critical 0000000180005d48     MSVCRT:utility.obj
 0002:00001d48       $unwind$atexit             0000000180005d48     MSVCRT:utility.obj
 0002:00001d50       $unwind$__GSHandlerCheckCommon 0000000180005d50     MSVCRT:gshandler.obj
 0002:00001d58       $xdatasym                  0000000180005d58     MSVCRT:amdsecgs.obj
 0002:00001d5c       $unwind$?dllmain_crt_process_attach@@YAHQEAUHINSTANCE__@@QEAX@Z 0000000180005d5c     MSVCRT:dll_dllmain.obj
 0002:00001d98       $unwind$?fin$0@?0??dllmain_crt_process_attach@@YAHQEAUHINSTANCE__@@QEAX@Z@4HA 0000000180005d98     MSVCRT:dll_dllmain.obj
 0002:00001d98       $unwind$?fin$0@?0??dllmain_crt_process_detach@@YAH_N@Z@4HA 0000000180005d98     MSVCRT:dll_dllmain.obj
 0002:00001d98       $unwind$?fin$1@?0??dllmain_crt_process_detach@@YAH_N@Z@4HA 0000000180005d98     MSVCRT:dll_dllmain.obj
 0002:00001da0       $unwind$?dllmain_crt_process_detach@@YAH_N@Z 0000000180005da0     MSVCRT:dll_dllmain.obj
 0002:00001df4       $unwind$?dllmain_dispatch@@YAHQEAUHINSTANCE__@@KQEAX@Z 0000000180005df4     MSVCRT:dll_dllmain.obj
 0002:00001e1c       $unwind$?filt$0@?0??dllmain_dispatch@@YAHQEAUHINSTANCE__@@KQEAX@Z@4HA 0000000180005e1c     MSVCRT:dll_dllmain.obj
 0002:00001e24       $unwind$__scrt_is_nonwritable_in_current_image 0000000180005e24     MSVCRT:utility.obj
 0002:00001e44       $unwind$__scrt_is_nonwritable_in_current_image$filt$0 0000000180005e44     MSVCRT:utility.obj
 0002:00001e4c       $unwind$__scrt_fastfail    0000000180005e4c     MSVCRT:utility_desktop.obj
 0002:00001e5c       $unwind$__report_gsfailure 0000000180005e5c     MSVCRT:gs_report.obj
 0002:00001e64       $unwind$capture_previous_context 0000000180005e64     MSVCRT:gs_report.obj
 0002:00001e70       $unwind$__security_init_cookie 0000000180005e70     MSVCRT:gs_support.obj
 0002:00001e7c       $unwind$__isa_available_init 0000000180005e7c     MSVCRT:cpu_disp.obj
 0002:00001e90       $xdatasym                  0000000180005e90     MSVCRT:guard_dispatch.obj
 0002:00001e98       $xdatasym                  0000000180005e98     MSVCRT:guard_xfg_dispatch.obj
 0002:00001ea0       .edata                     0000000180005ea0     GetStackTraceSuspendedStress.exp
 0002:00001ec8       rgpv                       0000000180005ec8     GetStackTraceSuspendedStress.exp
 0002:00001ed4       rgszName                   0000000180005ed4     GetStackTraceSuspendedStress.exp
 0002:00001ee0       rgwOrd                     0000000180005ee0     GetStackTraceSuspendedStress.exp
 0002:00001ee6       szName                     0000000180005ee6     GetStackTraceSuspendedStress.exp
 0002:00001f07       $N00001                    0000000180005f07     GetStackTraceSuspendedStress.exp
 0002:00001f14       $N00002                    0000000180005f14     GetStackTraceSuspendedStress.exp
 0002:00001f45       $N00003                    0000000180005f45     GetStackTraceSuspendedStress.exp
 0002:000023fc       .idata$6                   00000001800063fc     kernel32:KERNEL32.dll
 0002:00002456       .idata$6                   0000000180006456     vcruntime:VCRUNTIME140.dll
 0002:00002596       .idata$6                   0000000180006596     ucrt:api-ms-win-crt-string-l1-1-0.dll
 0002:000025b8       .idata$6                   00000001800065b8     ucrt:api-ms-win-crt-stdio-l1-1-0.dll
 0002:000025d8       .idata$6                   00000001800065d8     ucrt:api-ms-win-crt-runtime-l1-1-0.dll
 0003:00000000       ?UNNAMED_STR@?1??get_thread_name@@YAPEADPEAU_jvmtiEnv@@PEAUJNIEnv_@@PEAV_jobject@@@Z@4PEBDEB 0000000180007000     libGetStackTraceSuspendedStress.obj
 0003:00000058       ?GetVirtualThread_func@@3P6A?AW4jvmtiError@@PEAU_jvmtiEnv@@ZZEA 0000000180007058     libGetStackTraceSuspendedStress.obj
 0003:00000060       ?GetCarrierThread_func@@3P6A?AW4jvmtiError@@PEAU_jvmtiEnv@@ZZEA 0000000180007060     libGetStackTraceSuspendedStress.obj
 0003:00000068       agent_jvmti_env            0000000180007068     libGetStackTraceSuspendedStress.obj
 0003:00000070       agent_jni_env              0000000180007070     libGetStackTraceSuspendedStress.obj
 0003:00000078       current_agent_status       0000000180007078     libGetStackTraceSuspendedStress.obj
 0003:0000007c       ?i@@3HA                    000000018000707c     libGetStackTraceSuspendedStress.obj
 0003:00000080       jvmti_agent_thread         0000000180007080     libGetStackTraceSuspendedStress.obj
 0003:00000088       agent_thread_proc          0000000180007088     libGetStackTraceSuspendedStress.obj
 0003:00000090       agent_thread_arg           0000000180007090     libGetStackTraceSuspendedStress.obj
 0003:00000098       agent_data                 0000000180007098     libGetStackTraceSuspendedStress.obj
 0003:000000a8       ?event_mon@@3PEAU_jrawMonitorID@@EA 00000001800070a8     libGetStackTraceSuspendedStress.obj
 0003:000000b0       ?UNNAMED_LEN@?1??get_thread_name@@YAPEADPEAU_jvmtiEnv@@PEAUJNIEnv_@@PEAV_jobject@@@Z@4_KA 00000001800070b0     libGetStackTraceSuspendedStress.obj
 0003:000000b8       ?$TSS0@?1??get_thread_name@@YAPEADPEAU_jvmtiEnv@@PEAUJNIEnv_@@PEAV_jobject@@@Z@4HA 00000001800070b8     libGetStackTraceSuspendedStress.obj
 0003:000000c0       ?str@?1??TranslateState@@YAPEBDH@Z@4PADA 00000001800070c0     libGetStackTraceSuspendedStress.obj
 0003:000001f0       ?timeout@?1??agentProc@@YAXPEAU_jvmtiEnv@@PEAUJNIEnv_@@PEAX@Z@4_JA 00000001800071f0     libGetStackTraceSuspendedStress.obj
 0003:000001f8       ?g_tss_cv@@3U_RTL_CONDITION_VARIABLE@@A 00000001800071f8     MSVCRT:thread_safe_statics.obj
 0003:00000200       ?g_tss_event@@3PEAXEA      0000000180007200     MSVCRT:thread_safe_statics.obj
 0003:00000208       ?g_tss_mutex@@3U_RTL_CRITICAL_SECTION@@A 0000000180007208     MSVCRT:thread_safe_statics.obj
 0003:00000230       ?g_sleep_condition_variable_cs@@3P6AHPEAU_RTL_CONDITION_VARIABLE@@PEAU_RTL_CRITICAL_SECTION@@K@ZEA 0000000180007230     MSVCRT:thread_safe_statics.obj
 0003:00000238       ?g_wake_all_condition_variable@@3P6AXPEAU_RTL_CONDITION_VARIABLE@@@ZEA 0000000180007238     MSVCRT:thread_safe_statics.obj
 0003:00000244       ?__proc_attached@@3HA      0000000180007244     MSVCRT:dll_dllmain.obj
 0003:00000258       ?is_initialized_as_dll@@3_NA 0000000180007258     MSVCRT:utility.obj
 0003:00000259       ?module_local_atexit_table_initialized@@3_NA 0000000180007259     MSVCRT:utility.obj
 0003:00000260       ?module_local_atexit_table@@3U_onexit_table_t@@A 0000000180007260     MSVCRT:utility.obj
 0003:00000278       ?module_local_at_quick_exit_table@@3U_onexit_table_t@@A 0000000180007278     MSVCRT:utility.obj
 0003:000002a0       GS_ExceptionRecord         00000001800072a0     MSVCRT:gs_report.obj
 0003:00000340       GS_ContextRecord           0000000180007340     MSVCRT:gs_report.obj
